:020000040000FA
:04000000FA3060284A
:080008008612601C8616AE0092
:10001000030EAF008312051E21284008E0004108AE
:10002000E1004208E2004308E3004408E400450818
:10003000E5004608E6004708E700601C86166018E1
:100040008612051D2528BC0B21282830BC000F3046
:10005000A3008B100314851E031030193428B01828
:100060003828301839283A28E70CE60CE50CE40C5F
:10007000E30CE20CE10CE00C2F0E8300AE0E2E0E12
:02008000090075
:1000C000203084008001840A80300402031C6228EE
:1000D0002830BC008316FF3085051F308605C730E9
:1000E00087058312850186018701103083168E00F3
:1000F0008312703083168F0083120030031799002B
:100100000313003003179A000313003097000030E8
:100110009F00003083169F008312003003179E005B
:100120000313003003179F000313C73083168100A9
:10013000831230309000003092000030831694001B
:10014000831200309400A63083169800831200308A
:1001500083169B0083120030980033308316990079
:100160008312003083168C008312003083168D00BA
:10017000831210308B00B20BBB280130A400810128
:100180008E018F010B118B100B108C128C018D01C5
:100190008B1764000B190F211F21C9284808500232
:1001A000031DFE2849085102031DFE284A08520279
:1001B000031DFE284B085302031DFE284C08540261
:1001C000031DFE284D085502031DFE284E08560249
:1001D000031DFE284F085702031DFE285008C000CB
:1001E0005108C1005208C2005308C3005408C4009B
:1001F0005508C5005608C6005708C7004808D00073
:100200004908D1004A08D2004B08D3004C08D4005A
:100210004D08D5004E08D6004F08D70008000B1136
:10022000A40B08000430A4004521A30803191B29CE
:100230000613A303080006094039860008000310CE
:1002400087180314B40D34120C303402031D080057
:10025000B401061E3A293A08031D382931184D21E8
:10026000B118552131195F21B11977213508B9002D
:100270002030BA00BA03031007190314B80CB70CE6
:10028000B60CB50C0800331408000130871F043089
:10029000B1000310071FB10D08000030B000350891
:1002A000C800360AC900CE2008000130B000350869
:1002B000C800360AC9003808CA00CE20080002303B
:1002C000B0003508C800360AB200D801D901DA01F9
:1002D0000314D80DD90DDA0D0310B20B6929580893
:1002E000C9005908CA005A08CB00CE200800B91F1F
:1002F0007C29B51F08007E29B51B08000430B0001A
:100300003508C800360AB200D801D901DA01031451
:10031000D80DD90DDA0D0310B20B88293808CF009B
:10032000B51F9D29C901CA01CB015808CC00590845
:10033000CD005A08CE00CE200800CC01CD01CE0160
:100340005808C9005908CA005A08CB00CE20080036
:100350000708203A870008000708103A87000800BD
:080360000708083A87000800B5
:084000000800000000000800A8
:02400E00CC03E1
:00000001FF
